:02000000752960
:08000800FF0003088301FE0064
:100010000A08FD0000308A0091298030A100FE30DE
:100020009F2001309F207530A6003030B628A101F6
:10003000A117AE00FE309F202E089F28A401A90022
:10004000AA01A01124080319A0150530A300273028
:10005000A800103037200330A800E8303720A8016E
:1000600064303720A8010A30372029083E28A7002D
:100070002A08A6002908A500C5202508A500A30375
:100080000319A011240803194828230203184F2834
:100090002508031DA011A0194F28303E9F280800F5
:1000A000AC00861106118316861106110F308605E5
:1000B00083122C08A0187A283E30A6008030B62083
:1000C0003330AB008E201330A6008830B6208E204F
:1000D0006430B5208E206430B5202230AB008E20F5
:1000E000283079200C30792006307920A0142C0893
:1000F0007A282014AB00201C88280611033C031C1E
:100100008D288D200730A600D030B62003140800BB
:100110002014FE3C03199D280615201C201086156E
:100120000F3086052B08F039860400008611AB0ECF
:10013000000020188E283230B5202C08E128A11BA1
:1001400050280800AB00AB0DAB0D2B0D3839C13872
:100150009F00C830B5201F151F19AC281E08B2001B
:1001600083161E088312B100E128A601FC3EA500FB
:10017000A609031CC128FF300000A5070318BC28EE
:10018000A5070000A60FBB280800AA01A90110308E
:10019000AB00260DA90DAA0D2708A9022808031CEB
:1001A000280FAA020318DB282708A9072808031824
:1001B000280FAA070310A50DA60DAB0BC92825080B
:1001C000E128831383120313080038083406BF00A4
:1001D000BF1B1A29B81B032937083302031C00343C
:1001E000031D013438083402031C0034031D01349C
:1001F00039083502031C0034031D01343A08360265
:10020000031C0034013433083702031C0034031D7F
:10021000013434083802031C0034031D013435084E
:100220003902031C0034031D013436083A02031C52
:1002300000340134B41F01340034B501B6019630E6
:10024000BE00C013B61F3029B609B509B409B309F9
:10025000B30F2F29B40F2F29B50A0319B60AC017F7
:10026000B60803194B293D1F4229B61F4229B40F76
:100270004229B50F4229B60F42290314B60CB50C1A
:10028000B40CBE0A0830BE073408B3003508B40009
:100290003608B5006029B508031D60290830BE0284
:1002A0003408031D5C290830BE023308031D5B2996
:1002B0003608BE006A29B301B5003308B400B301A3
:1002C000B51B68290310B30DB40DB50DBE0360292D
:1002D000C01FB5133308B6003E08B3003508BE0092
:1002E0003408B5003E08B400E1284030BD00A0014C
:1002F00083168113FF309C009F01DD3085000130A3
:1003000086008312C50160309F008E3083169F00E7
:1003100088308100831281018B168B178A110A1293
:10032000A229013045028A110A12031D9A29C60A20
:100330000319C70A0B117D088A007E088300FF0E8F
:100340007F0E0900851485128A110A1287195E2A08
:100350008A110A12871DA82900308A01A2203108BB
:10036000B3003208B4008A011D213608C4003508E4
:10037000C3003408C2003308C1008A110A12C21B2C
:10038000C729883041028A110A120318AC29D70103
:100390000B3057028A110A1203181D2AC601C70121
:1003A00000308A01A2203108B3003208B4008A016B
:1003B0001D213608C4003508C3003408C2003308C4
:1003C000C100B601B501B4018830B3004408BA00D9
:1003D0004308B9004208B8004108B7008A01E52087
:1003E000013C8A110A120319D0290130C5000030DE
:1003F0008A01A2203108B3003208B4008A011D210D
:100400003608C4003508C3003408C2003308C100F0
:100410008A110A12C21B122A883041028A110A125A
:100420000318F729C5015708483E84004608800094
:10043000D70A8A110A12031DC8298A010D208030AB
:10044000A1008A01172048088A011E2020308A0155
:10045000502049088A011E2020308A0150204A0875
:100460008A011E2020308A0150204B088A011E205C
:1004700020308A0150204C088A011E208030A100C3
:10048000C0308A0117204D088A011E2020308A01C1
:1004900050204E088A011E2020308A0150204F082B
:1004A0008A011E2020308A01502050088A011E2017
:1004B00020308A01502051088A011E208A01A22979
:0404C0008A01602A23
:02400E00323F3F
:00000001FF
